:020000040800F2
:1000000000100020991C00081D1C00081F1C00087F
:10001000211C0008231C0008251C0008000000000B
:10002000000000000000000000000000271C000885
:10003000291C0008000000002B1C00082D1C0008D3
:10004000E11C0008E11C0008E11C0008E11C00089C
:10005000E11C0008E11C0008E11C0008E11C00088C
:10006000E11C0008E11C0008E11C0008E11C00087C
:10007000E11C0008E11C0008E11C0008E11C00086C
:10008000E11C0008E11C0008E11C00080000000061
:10009000000000000000000000000000E11C00085B
:1000A000E11C0008E11C0008E11C0008E11C00083C
:1000B000E11C0008E11C0008E11C0008E11C00082C
:1000C000E11C00080000000000000000E11C000826
:1000D000E11C0008311C0008E11C0008E11C0008BC
:1000E000E11C0008E11C0008E11C00080000000001
:1000F0000000000000000000000000000000000000
:1001000000000000000000000000000000000000EF
:100110000000000000000000E11C00083D1C000879
:1001200000000000000000000000000000000000CF
:1001300000000000000000000000000000000000BF
:1001400000000000000000000000000000000000AF
:10015000000000000000000000000000000000009F
:10016000000000000000000000000000000000008F
:10017000000000000000000000000000000000007F
:10018000000000000000000000000000000000006F
:10019000000000000000000000000000000000005F
:1001A000000000000000000000000000000000004F
:1001B000000000000000000000000000000000003F
:1001C0000000000000000000000000005FF808F1DF
:1001D00010B5054C237833B9044B13B10448AFF381
:1001E00000800123237010BD780000200000000073
:1001F000F42D000808B5034B1BB103490348AFF3C6
:10020000008008BD000000007C000020F42D0008E4
:10021000D0400B1CD1409C46203AD3401843524258
:10022000634693401843704738B50E4B054618781F
:100230004FF47A73B3FBF0F30B4A1068B0FBF3F0A2
:1002400000F098F8044658B90F2D09D802462946FF
:100250004FF0FF3000F04EF8044B20461D6038BDD3
:10026000012038BD000000200C0000200400002008
:1002700008B5032000F02CF80020FFF7D5FF01F0AF
:100280005BFC002008BD0000034A044B11681B788A
:100290000B441360704700BFD00000200000002016
:1002A000014B1868704700BFD000002038B50446E5
:1002B000FFF7F6FF0546631C1EBF044B1B78E418CE
:1002C000FFF7EEFF401B8442FAD838BD0000002043
:1002D000074A0002D36800F4E06023F4E0631B04E3
:1002E0001B0C43F0BF6343F400330343D3607047F8
:1002F00000ED00E0174B30B5DC68C4F30224C4F114
:100300000703251D042B28BF0423062D4FF00105EC
:1003100098BF002405FA03F303F1FF3388BF033CC1
:100320001940A14005FA04F4013C2240002842EAA9
:1003300001024FEA0212AFBF00F16040064B00F02D
:100340000F00D2B2A5BFD2B200F561401A5480F8B6
:10035000002330BD00ED00E014ED00E00123420970
:1003600000F01F0003FA00F0014B43F82200704731
:1003700000E100E00138B0F1807F0AD2F021064BA5
:10038000064A586082F823100020072298601A60FD
:1003900070470120704700BF10E000E000ED00E072
:1003A00090F8213010B5022B03D004238363012081
:1003B00010BD03681A6822F00E021A601A6822F053
:1003C00001021A60184A93421FD0143293421ED081
:1003D000143293421DD0143293421DD014329342F2
:1003E0001DD0143293420CBF4FF480134FF0807332
:1003F0000E4A00245360012380F82130436B80F8BB
:1004000020407BB19847204610BD0123F0E7102320
:10041000EEE74FF48073EBE74FF48053E8E74FF4D7
:100420008033E5E7184610BD080002400000024096
:10043000114AD36813F0100305D01049CB6943F07B
:100440000203CB611023D268500706D50B4943F055
:100450000403CA6942F00102CA61074AD169C907A7
:1004600008D50648C16941F00401C161D16921F094
:100470000101D161D360704700200240D800002004
:10048000064B186910F0800007D0054A5A6002F147
:1004900088325A601869C0F3C010704700200240CB
:1004A00023016745034A0020136943F08003136169
:1004B000704700BF00200240F8B50646FFF7F0FE87
:1004C000114C07462546E368D80712D4E36899061D
:1004D00044BF2023E360EB68DA0606D4EB69DB0750
:1004E00003D4E86810F0040002D0FFF7A1FF012058
:1004F000F8BD731CE7D00EB90320F8BDFFF7D0FE9E
:10050000C01B8642DFD2F7E7002002402DE9F84FFA
:100510001F4C9946237E0546012B0F46904633D04B
:1005200001234CF250302376FFF7C6FF40BB012D6C
:1005300003D0022D0CBF022504250026B246DFF8A9
:1005400054B0320140464946FFF762FEC4F81CA091
:10055000DBF8103080B243F00103CBF8103027F8FD
:1005600016004CF25030FFF7A7FFDBF8103023F0F5
:100570000103CBF8103018B90136F3B29D42E0D830
:1005800000232376BDE8F88F0220BDE8F88F00BF76
:10059000D8000020002002400022064BDA61064B02
:1005A0001A6942F004021A611A6942F040021A61A3
:1005B000704700BFD8000020002002400022064BF8
:1005C000DA61064B1A6942F002021A6158611A692F
:1005D00042F040021A617047D8000020002002401B
:1005E0002DE9F041234D07462B7E8846012B3DD057
:1005F000012403682C76022B4CF2503013D1FFF704
:100600005BFF20B1012000232B76BDE8F081FFF7CE
:10061000C3FF4CF25030FFF74FFF174A136923F026
:1006200004031361EFE7FFF747FF0028EAD14FF01B
:10063000FF33C8F800302046BE680F4CFA68BB682C
:1006400003EB82239E42DED23046FFF7B7FF4CF227
:100650005030FFF731FF236923F00203236110B10B
:10066000C8F80060CFE706F58066E7E70220BDE83E
:10067000F08100BFD8000020002002402DE9F74F94
:1006800000221646654BDFF8A4E1DFF8A4C14FF065
:1006900001080C6808FA06F808EA0404A0457FD1AE
:1006A0004D68122D00F0AF8000F28880022D00F01E
:1006B000A7807CD8002D00F08E80012D00F09E8058
:1006C0004FF00F09FF2C93BF824606F18045083D8D
:1006D000D0F800B092BFB500D0F804B0AD0009FA70
:1006E00005F82BEA080802FA05F588BF00F1040AAC
:1006F00048EA0505CAF80050D1F804A01AF0805F56
:100700004ED0474D464FAD6926F0030845F0010530
:10071000BD61BD6908F1804805F00105019508F546
:10072000803806F0030B019D4FEA8B0BD8F8085078
:1007300009FA0BF925EA09093A4DA84268D005F5EE
:100740008065A84266D005F58065A84264D005F5AD
:100750008065A8420CBF0325042505FA0BF545EA80
:100760000905C8F808501D681AF4803F14BF2543D6
:10077000A5431D605D681AF4003F14BF2543A543DF
:100780005D609D681AF4801F14BF2543A5439D60DA
:10079000DD681AF4001F14BF2C4325EA0404DC6052
:1007A0000136102E7FF473AF03B0BDE8F08F032D38
:1007B00022D0112D84D1CA68043281E71A4FBD427C
:1007C00009D012D8DFF86C904D4504D009F5803976
:1007D0004D457FF475AF8A68C2B1012A0CBFC0F8DD
:1007E0001080C0F8148008226AE77545F3D065458B
:1007F000F1D0DFF84490EBE7002261E7CA685FE7D9
:10080000CA6808325CE7CA680C3259E7042257E725
:100810000025A2E70125A0E702259EE7000401408C
:1008200000100240000801400000211000003110BB
:100830000000321000001110000022100AB1016106
:1008400070470904FBE7C3685940C1607047000066
:1008500003682DE9F341DB07054610D42B689F0799
:100860005ED42B68190700F195802B685A0700F1B8
:10087000BF80EA69002A40F02D81002014E0904CEE
:10088000636803F00C03042B07D0636803F00C03C8
:10089000082B0CD16368DE0309D523689C03DDD5E2
:1008A0006B68002BDAD1012002B0BDE8F0816B68E3
:1008B000B3F5803F10D1236843F480332360FFF702
:1008C000EFFC064623689803C8D4FFF7E9FC801BB9
:1008D0006428F7D90320E7E79BB9236823F4803322
:1008E0002360236823F480232360FFF7D9FC0646A6
:1008F00023689903B2D5FFF7D3FC801B6428F7D98E
:10090000E8E7B3F5A02F236803D143F480232360E5
:10091000D1E723F480332360236823F48023CDE7D9
:10092000674C636813F00C0F07D0636803F00C0387
:10093000082B10D16368DA030DD423689B0702D516
:100940002B69012BAFD123686A6923F0F80343EACE
:10095000C203236085E72A695A4B6AB101221A60F3
:10096000FFF79EFC064623689F07ECD4FFF798FC30
:10097000801B0228F7D9ADE71A60FFF791FC064605
:10098000236898077FF56DAFFFF78AFC801B02286C
:10099000F6D99FE7AA694A4C4B4BDAB101221A609B
:1009A000FFF77EFC0646636A9B070DD54FF4FA52AB
:1009B000464B1B68B3FBF2F3019300BF019B5A1E29
:1009C0000192002BF9D150E7FFF76AFC801B022847
:1009D000E9D97FE71A60FFF763FC0646636A9F0761
:1009E0007FF543AFFFF75CFC801B0228F6D971E767
:1009F000334CE369D80024D40127E36943F08053E2
:100A0000E361E36903F080530093009B304E336849
:100A1000D90518D5EB68012B26D1236A43F00103D1
:100A20002362FFF73DFC41F288368046236A9B072C
:100A30003FD5002F3FF41DAFE36923F08053E361FE
:100A400017E70027E2E7336843F480733360FFF76A
:100A500027FC80463368DA05DCD4FFF721FCA0EBE5
:100A600008006428F6D935E7ABB9236A41F2883823
:100A700023F001032362236A23F004032362FFF7B8
:100A80000FFC0646236A9807D3D5FFF709FC801BA5
:100A90004045F7D91EE7052B236A03D143F0040331
:100AA0002362BAE723F001032362236A23F00403DD
:100AB000B6E7FFF7F5FBA0EB0800B042B6D909E7AF
:100AC0000010024000004242800442420C0000201C
:100AD00000700040224C636803F00C03082B3FF4C5
:100AE000E2AE00231F4E022A33602BD1FFF7D8FB62
:100AF0000746236899011FD42B6AB3F5803F05D1BF
:100B0000E26AA96822F00F020A43E262696A626837
:100B10000B4322F474121343636001233360FFF725
:100B2000BFFB054623689A013FF5A7AEFFF7B8FB68
:100B3000401B0228F6D9CDE6FFF7B2FBC01B022806
:100B4000D7D9C7E6FFF7ACFB054623689B017FF5C5
:100B500094AEFFF7A5FB401B0228F6D9BAE600BF0A
:100B6000001002406000424230B589B06C461B4B19
:100B700003F11005224618685968083303C2AB42D6
:100B80001446F7D1164B04AC03F110052246186841
:100B90005968083303C2AB421446F7D111494B6878
:100BA00003F00C02082A17D1C3F3834208A80244B9
:100BB000DB0312F8202C0CD5CB6A0B4803F00F0393
:100BC000504308AA134413F8103CB0FBF3F009B0EB
:100BD00030BD06485043FAE70348F8E70C2E0008FA
:100BE0001C2E00080010024000127A0000093D008F
:100BF0000268F8B512F0020F05463C4C11D05707B9
:100C000042BF636843F4E0636360160742BF6368F2
:100C100043F4605363606368816823F0F0030B431F
:100C20006360D0071AD42A68510756D4130706D533
:100C300063682A6923F4605343EAC2036360FFF7E1
:100C400093FF63682A4AC3F30313D35CD840294B4C
:100C500018600020FFF7E8FA0020F8BD68682368F4
:100C6000012802D19A0305D4F8BD02281BD113F044
:100C7000007F39D0636841F2883723F003031843BB
:100C80006060FFF70DFB6B680646012B0ED16368B1
:100C900003F00C03042BC6D0FFF702FB801BB84205
:100CA000F5D90320F8BD13F0020FE2E7022B0FD1B4
:100CB000636803F00C03082BB5D0FFF7F1FA801B33
:100CC000B842F5D9EDE7FFF7EBFA801BB842E8D858
:100CD000636813F00C0FF6D1A5E76368E96823F4A5
:100CE000E0630B436360A1E70120F8BD0010024000
:100CF0001A2F00080C000020044B054A5B68C3F360
:100D00000223D35C034A1068D840704700100240A9
:100D10002A2F00080C000020044B054A5B68C3F32F
:100D2000C223D35C034A1068D840704700100240C9
:100D30002A2F00080C00002003680020DA6842F027
:100D40000102DA601A6842F001021A6070477047C7
:100D5000704770477047036810B51A6904469107D9
:100D60000ED5DA6892070BD56FF002021A610122E4
:100D70009B6902779B0777D0FFF7EAFF0023237771
:100D800023681A69500710D5DA6851070DD56FF03E
:100D900004021A6102229B69227713F4407F2046E5
:100DA00068D0FFF7D5FF0023237723681A6912075D
:100DB0000FD5DA6810070CD56FF008021A6104220B
:100DC000DB692277990720465AD0FFF7C1FF00233D
:100DD000237723681A69D20610D5DA68D0060DD5B4
:100DE0006FF010021A610822DB69227713F4407F4A
:100DF00020464BD0FFF7ACFF0023237723681A6906
:100E0000D10708D5DA68D20705D56FF00102204670
:100E10001A6100F0F1FB23681A69100608D5DA6838
:100E2000110605D56FF0800220461A6100F0C5F862
:100E300023681A69520608D5DA68500605D56FF09E
:100E4000400220461A61FFF785FF23681A69910660
:100E500022D5DA6892061FD56FF020022046BDE841
:100E600010401A6100F0A8B8FFF771FF2046FFF7A5
:100E700070FF83E7FFF76BFF2046FFF76AFF92E7FB
:100E8000FFF765FF2046FFF764FFA0E7FFF75FFF6E
:100E90002046FFF75EFFAFE710BD0000264A03685B
:100EA00090420AD0B0F1804F07D0A2F59432904220
:100EB00003D002F58062904211D14A6823F070039A
:100EC00013431D4A904215D0B0F1804F12D0A2F5C5
:100ED000943290420ED002F5806290420AD0174AB6
:100EE000904207D002F58062904203D002F5806202
:100EF000904203D1CA6823F4407313434A6923F034
:100F00008003134303608B68C3620B6883620A4BE0
:100F100098420BD003F5A053984207D003F58063A5
:100F2000984203D003F58063984201D10B690363B3
:100F300001234361704700BF002C01400040014085
:100F400010B50446A0B190F83D3003F0FF021BB984
:100F500080F83C2000F012FE0223206884F83D3027
:100F6000211DFFF79BFF0123002084F83D3010BDB9
:100F7000012010BD90F83C3010B5012B4FF002035A
:100F800018D080F83D3003680C685A68496822F030
:100F900070025A605A6822435A609A6822F08002AE
:100FA0009A609A680A439A60012380F83D300023D2
:100FB00080F83C30184610BD704770470368DA6807
:100FC00022F49072DA605A6922F001025A612023F9
:100FD00080F83A30704700002DE9F04781460568F7
:100FE000C2682B69C16923F4405313432B618368A2
:100FF0000069EA680343D9F8140022F41642034357
:1010000022F00C020B431343EB606B69D9F81820F4
:1010100023F440731343B1F5004F6B617E4B7FD1D6
:101020009D424FF0190447D1FFF776FE04FB00F311
:10103000D9F804704FF064087F00B3FBF7F3B3FBFB
:10104000F8F31F01FFF768FE6043D9F804305B0036
:10105000B0FBF3F6FFF760FE6043D9F804305B00A5
:10106000B0FBF3F3B3FBF8F308FB1363DB0032339D
:10107000B3FBF8F35B0003F4F876FFF74DFE604333
:10108000D9F804205200B0FBF2FAFFF745FE6043A6
:10109000D9F804305B00B0FBF3F3B3FBF8F308FBC3
:1010A00013A3DB003233B3FBF8F303F007033B4435
:1010B0003344AB60BDE8F087FFF71EFE04FB00F38E
:1010C000D9F804704FF064087F00B3FBF7F3B3FB6B
:1010D000F8F31F01FFF710FE6043D9F804305B00FE
:1010E000B0FBF3F6FFF708FE6043D9F804305B006D
:1010F000B0FBF3F3B3FBF8F308FB1363DB0032330D
:10110000B3FBF8F35B0003F4F876FFF7F5FD6043FB
:10111000D9F804205200B0FBF2FAFFF7EDFDB6E774
:101120009D424FF0190443D1FFF7F6FD04FB00F395
:10113000D9F804604FF06408B600B3FBF6F3B3FBD4
:10114000F8F31E01FFF7E8FD6043D9F804309B0077
:10115000B0FBF3F7FFF7E0FD6043D9F804309B00E4
:10116000B0FBF3F3B3FBF8F308FB13731B0132334B
:10117000B3FBF8F303F0F007FFF7CEFD6043D9F8B7
:1011800004209200B0FBF2FAFFF7C6FD6043D9F8E5
:1011900004309B00B0FBF3F3B3FBF8F308FB13A39D
:1011A0001B013233B3FBF8F303F00F033B437FE73C
:1011B000FFF7A2FD04FB00F3D9F804604FF06408C8
:1011C000B600B3FBF6F3B3FBF8F31E01FFF794FD93
:1011D0006043D9F804309B00B0FBF3F7FFF78CFDB8
:1011E0006043D9F804309B00B0FBF3F3B3FBF8F392
:1011F00008FB13731B013233B3FBF8F303F0F00762
:10120000FFF77AFD6043D9F804209200B0FBF2FAB0
:10121000FFF772FDBAE700BF00380140F8B5044699
:101220000E4617461D4621680B6836EA030301D1B6
:101230000020F8BD6B1CF7D095B923680320DA684D
:1012400022F4D072DA605A6922F001025A61202336
:1012500084F8393084F83A30002384F83830F8BD07
:10126000FFF71EF8C01B8542DDD2E6E710B5044645
:1012700040B390F8393003F0FF021BB980F83820F2
:1012800000F090FC2423226884F83930D36820468B
:1012900023F40053D360FFF79FFE236800201A69F0
:1012A00022F490421A615A6922F02A025A61DA68DD
:1012B00042F40052DA602023E06384F8393084F885
:1012C0003A3010BD012010BD2DE9F0411F4690F8C5
:1012D00039300446202B0D4690464ED1002949D086
:1012E000002A47D090F83830012B46D0012380F8EF
:1012F00038300023C363212380F83930FEF7D0FF54
:101300000646A4F82480A4F82680E38C9BB26BB92F
:101310003B46324640212046FFF780FFA8B92023F4
:1013200084F8380084F83930BDE8F081E38C324627
:10133000013B9BB2E384A3688021B3F5805F204624
:101340003B460ED1FFF76AFF10B10320BDE8F081E4
:101350002B882268C3F308035360236943B902351D
:10136000D3E7FFF75BFF0028EFD123682A785A60A4
:101370000135CAE70120BDE8F0810220BDE8F08117
:1013800090F83A30202B20D1E9B1E2B190F8383012
:10139000012B1AD0C285828500232222C36380F8E4
:1013A0003A2002688162D16880F8383041F4807157
:1013B000D1605169184641F001015161D16841F095
:1013C0002001D160704701207047022070477047AC
:1013D00090F83A3010B5222B36D183680169B3F505
:1013E000805F0268836A23D15268E9B9C2F30802B8
:1013F00023F8022B8362C48D013CA4B2C4858CB94E
:101400000368DA6822F02002DA60DA6822F4807277
:10141000DA605A6922F001025A61202380F83A30DA
:1014200000F0CAF8002010BDD2B223F8012BE1E78A
:1014300021B9591C526881621A70DCE75268591C44
:10144000816202F07F02F7E7022010BD70470000C2
:10145000036870B51A6804461607D9685D6907D134
:1014600096065AD58D0658D5BDE87040FFF7B0BF37
:1014700015F0010502D111F4907F4ED0D30705D5A8
:10148000CE0542BFE36B43F00103E363500704D58D
:101490001DB1E36B43F00203E363930704D51DB171
:1014A000E36B43F00403E363160704D51DB1E36B5C
:1014B00043F00803E363E36B002B66D0950604D585
:1014C000880602D52046FFF783FF236820465D6922
:1014D000E26B110702D415F040051AD0FFF76EFD3C
:1014E00023685A69520610D55A69606B22F040028F
:1014F0005A6150B1254B4363FEF752FF002844D098
:10150000606BBDE87040436B18472046FFF79EFFB5
:1015100070BDFFF79BFFE56370BD160627D50D066E
:1015200025D594F83920212A2FD1A268B2F5805F01
:10153000226A17D11188C1F308015960216979B96C
:1015400002322262E28C013A92B2E284EAB9DA68AB
:1015500022F08002DA60DA6842F04002DA6070BDA0
:101560000132EEE7511C216212785A60EAE7500618
:101570000BD54A0609D5DA68204622F04002DA6027
:10158000202384F83930FFF722FF70BD9115000841
:1015900008B50023406AC385C384FFF757FF08BD21
:1015A00008B5FEF76DFF3422024BDA60BDE8084053
:1015B000FEF778BF0020024002680A4B9A420FD122
:1015C000094A0A49136808780949C8540133632B4A
:1015D00088BF00230549136006480122FFF7D0BEEB
:1015E000704700BF00380140B8000020C000002054
:1015F00088010020FC0000200268084B9A420BD1B1
:10160000074A136801331360064A136801331360F5
:10161000054A136801331360704700BF001400408F
:10162000B0000020A8000020A40000200A460A23E1
:1016300001460148FFF748BEFC00002010B51446E3
:101640000A230248FFF740FE204610BDFC000020A0
:101650002DE9F041002407462646104DDFF8408072
:10166000BB78023B9C4202DB3046BDE8F0813B196F
:10167000DA781B79296802EB032292B20023012059
:10168000FEF744FF18B1404600F0CCFB01262B6862
:10169000023402332B60E4B2E2E700BF080000200E
:1016A0006C2E0008002373B5164D174C2B60174B9A
:1016B0000646AB603F23EB60E36923F02003E36160
:1016C000FEF7DEFE124B1A784AB90122114928466C
:1016D0001A70FEF785FF10B10F4800F0A3FB3046EB
:1016E000FFF7B6FF0546FEF7DDFE2846E36943F047
:1016F0002003E361E36903F020030193019B02B03F
:1017000070BD00BF9400002000100240004000089F
:10171000B4000020AC000020782E000870B5064C04
:10172000064E074D227821463046013400F006FB74
:10173000AC42F7D170BD00BF004000085E2E00082B
:1017400010400008B0B50D4A00AFD3690C4823F033
:101750002003D36100F066FB0A4B0B4A1B680B4C5D
:101760000B481360236000F05DFB0A4B1B6883F39A
:1017700008882368BD46BDE8B04018470010024005
:10178000872E0008044000083C010020840100204E
:10179000992E00080040000873B50446254BA17837
:1017A00018681B7900908DF8043063185A78601C13
:1017B00000F0A5F901280BD000231F4EA2785D1C74
:1017C0000232DBB29A422FDA1C4800F02BFB0CE00D
:1017D00011238DF801306378DD2B01D0EE2B07D17A
:1017E0002046FFF75FFF012802D122238DF8013048
:1017F0009DF802100DF1010000F066F963788DF894
:101800000300EE2B08D00A2B06D09DF80210684684
:101810000331C9B2FFF70AFF6378EE2B02D1084803
:1018200000F000FB02B070BDE15C304600F086FACB
:101830002B46C3E72C2E0008362E00083C2E00084D
:101840004D2E000810B590B02822002106A800F007
:101850006DFA1422002101A800F068FA01230A930E
:10186000102302240B934FF4002306A80F93069431
:101870000D94FEF7EDFF0F23002101934FF48063D9
:1018800001A80294039104930591FFF7B1F910B0F8
:1018900010BD00002DE9F047C8B008AFFF220021BD
:1018A000384600F043FA734B002418681B79029005
:1018B0008DF80C30FEF7DCFCFFF7C4FF102200218E
:1018C0000DEB020000F032FA6B4B4FF400419A69C5
:1018D0006A4842F010029A619A694FF0010802F0DA
:1018E00010020092009A9A69654D42F004029A61D2
:1018F0009B69002203F004030193019BFEF79EFF06
:101900004FF400430493022304A95C48CDF81480EB
:1019100007930694FEF7B2FE4FF4E133594A284686
:1019200085E80C000C23AC606B61EC602C61AC6151
:10193000EC61FFF79BFC40F23F63534E5349304646
:1019400086E80A000923B460F360B4610494059446
:10195000FFF7F6FA04A9304604940594FFF70AFB52
:10196000224621462520FEF7C5FC2520FEF7F6FC81
:10197000224621463720FEF7BDFC3720FEF7EEFC5D
:101980003046FFF7D9F9424641492846FFF7F8FCAF
:10199000404B21461B68404E986800F04BFA3F4888
:1019A00000F040FA3E4800F03DFA3E4A3E493F48CA
:1019B00000F0C4F93E4800F035FA384800F032FA39
:1019C000FFF7EEFDFFF7AAFE9DF80A100DF10900E2
:1019D00000F07AF88DF80B006420FEF767FC9DF8A4
:1019E0000A1002A80331C9B2FFF720FE2546B1460E
:1019F000DFF8888040F6B83332689A4201D9FFF7A1
:101A0000A1FE2C4A2C4B11681B6899421ED02B4C0E
:101A1000481C615C6B1C79550021DBB21D466328B4
:101A2000106088BF1160264A1160254B1B68642B2B
:101A30001ED900253846FFF7AFFE64220021384644
:101A400000F074F92C46C9F8005001E0002CECD1EC
:101A5000DFF870A0DAF80030B3F5FA7FCAD94FF496
:101A600000414046FEF7EFFE0023CAF80030C1E710
:101A70000124EDE7312E0008001002400010014063
:101A8000FC00002000380140440100200014004008
:101A9000C000002010000020A40000209F2E00089D
:101AA000C92E0008D62E0008DF2E0008EB2E0008F5
:101AB000FC2E0008BC000020B80000208801002097
:101AC000B0000020A800002010B5FF230446221A11
:101AD000D2B2914201D8184610BD14F8012B5340E0
:101AE000082213F0800F02F1FF324FEA430318BFC0
:101AF00083F0310312F0FF02DBB2F2D1E7E730B539
:101B0000FF2305462C1AE4B2A14203D89B1A58427F
:101B1000584130BD15F8014B6340082413F0800F85
:101B200004F1FF344FEA430318BF83F0310314F08C
:101B3000FF04DBB2F2D1E5E70E4B82B09A6942F0C6
:101B400001029A619A6902F001020092009ADA6930
:101B500042F08052DA61DB69074A03F08053019357
:101B6000019B536823F0E06343F08063536002B04D
:101B7000704700BF00100240000001400268084B9F
:101B800082B09A420AD103F5FE33DA6942F02002AC
:101B9000DA61DB6903F020030193019B02B0704717
:101BA0000014004010B5044686B01022002102A89F
:101BB00000F0BCF82268174B9A4228D103F558432D
:101BC0009A6902A942F480429A619A69124802F421
:101BD00080420092009A9A6942F004029A619B69DD
:101BE00003F004030193019B4FF40073029302235B
:101BF000039303230593FEF741FD4FF480630293A3
:101C0000002302A9044803930493FEF737FD06B0AE
:101C100010BD00BF00380140000801407047FEE7DA
:101C2000FEE7FEE7FEE7704770477047FEF72CBB04
:101C30000148FFF70DBC00BFFC0000200148FFF782
:101C40008AB800BF44010020104B1A6842F001021C
:101C50001A6059680E4A0A405A601A6822F0847263
:101C600022F480321A601A6822F480221A605A68BC
:101C700022F4FE025A604FF41F029A600022DA62D8
:101C80004FF00062034B9A60704700BF00100240A3
:101C90000000FFF800ED00E0002103E00B4B5B5873
:101CA000435004310A480B4B42189A42F6D30A4A71
:101CB00002E0002342F8043B084B9A42F9D3FFF7B5
:101CC000C3FF00F00FF8FFF7E5FD7047D42F0008C1
:101CD0000000002074000020780000208C0200200A
:101CE000FEE7000070B500250C4E0D4CA41BA4109F
:101CF000A54209D101F07EF800250A4E0A4CA41B2A
:101D0000A410A54205D170BD56F82530984701357D
:101D1000EEE756F8253098470135F2E7CC2F00085A
:101D2000CC2F0008CC2F0008D02F00080346024417
:101D3000934200D1704703F8011BF9E70FB40A4B37
:101D400013B51C6824B1A36913B9204600F0DAFA70
:101D500005AB049AA1682046019300F09BFC02B0F9
:101D6000BDE8104004B070471000002070B50E466A
:101D7000054618B183690BB900F0C4FAAB69AC68C9
:101D800013B9284600F0BEFA234B9C4217D16C6869
:101D9000A3891B071DD52369DBB1013EA36816F893
:101DA000011F013BA360E9B9002B2EDA22460A216C
:101DB000284600F0F5F8013011D00A2070BD174B0D
:101DC0009C4201D1AC68E3E7154B9C4208BFEC682C
:101DD000DEE72146284600F035F90028DDD04FF037
:101DE000FF3070BD002B04DAA269934206DB0A299A
:101DF00004D023685A1C22601970CFE72246284677
:101E000000F0CEF80130C9D1E9E70A2023685A1C56
:101E10002260187070BD00BF582F0008782F00088E
:101E2000382F0008024B01461868FFF79FBF00BF1C
:101E30001000002000294FF480630CBF0222002212
:101E400000F000B82DE9F7431D46514B04461E68CB
:101E50000F46904626B1B36913B9304600F052FAE6
:101E60004C4B9C4252D17468B8F1020F06D0B8F1C5
:101E7000010F00F28980002DC0F286802146304695
:101E800000F0D6F9616B41B104F14403994202D0EC
:101E9000304600F02DFB002363630023A3616360E1
:101EA000A3891B0603D52169304600F021FBA389D5
:101EB000B8F1020F23F44A6323F00303A3815DD03A
:101EC00001AB6A462146304600F0A6FAA3891843C2
:101ED000A0812DBB009D284600F002FB074600288C
:101EE0004ED1DDF80090A9453CD14FF0FF30A389D9
:101EF00043F00203A3810023A36004F1470323609E
:101F000023610123636103B0BDE8F083224B9C424F
:101F100001D1B468A8E7214B9C4208BFF468A3E74D
:101F2000002FD8D0B36913B9304600F0EBF9B8F1FF
:101F3000010F08BFA389276004BF43F00103A381F9
:101F4000A389276113F0080065611BD013F001001D
:101F50004FF000031FBF6D42A360A561184608BF84
:101F6000A560D0E7484600F0BBFA07460028BCD081
:101F7000A3894D4643F08003A381D3E70020B6E751
:101F8000A946F5E7A060BEE74FF0FF30BBE700BF12
:101F900010000020582F0008782F0008382F000864
:101FA000F8B50E461446054618B183690BB900F022
:101FB000A9F9214B9C422AD16C68A369A360A3892B
:101FC0001A072ED5236963B323692068F6B2C01AB5
:101FD00063693746984204DB2146284600F028F919
:101FE00028BBA3680130013BA36023685A1C226010
:101FF0001E706369984204D0A389DB0719D50A2EA5
:1020000017D12146284600F013F990B10FE00B4B91
:102010009C4201D1AC68D0E7094B9C4208BFEC68F8
:10202000CBE72146284600F00DF80028CCD04FF031
:10203000FF373846F8BD00BF582F0008782F00083A
:10204000382F0008324B70B51D6806460C4625B186
:10205000AB6913B9284600F055F92E4B9C420FD1BD
:102060006C68B4F90C309AB215072CD4D00611D490
:102070000922326043F04003A3814FF0FF3070BD6E
:10208000254B9C4201D1AC68EBE7244B9C4208BF36
:10209000EC68E6E7510712D5616B41B104F14403E6
:1020A000994202D0304600F023FA00236363A389EB
:1020B00023F02403A3810023636023692360A389A1
:1020C00043F00803A38123694BB9A38903F4207368
:1020D000B3F5007F03D02146304600F0C1F9A28954
:1020E00012F001030CD00023A36063695B42A3617B
:1020F000236953B9B4F90C3013F08000BAD170BD24
:10210000920758BF6369A360F2E70020F7E700BFBA
:1021100010000020582F0008782F0008382F0008E2
:102120008A892DE9F041054610070C465AD44B68C0
:10213000002B05DC0B6C002B02DC0020BDE8F081DD
:10214000E66A002EF9D0002312F480522F682B602B
:1021500033D0606DA3895A0705D56368C01A636BD5
:102160000BB1236CC01A00230246E66A216A284696
:10217000B047431CA38906D129681D294BD82B4A97
:10218000CA40D60747D5002262602269D90422607E
:1021900004D5421C01D12B6803B96065616B2F60C7
:1021A0000029CAD004F14403994202D0284600F025
:1021B0009FF900206063BDE8F081216A0123284671
:1021C000B047411CC6D12B68002BC3D01D2B01D0BA
:1021D000162B01D12F60B0E7A38943F04003A38100
:1021E000BDE8F0810F69002FA7D0930718BF002327
:1021F0000E6808BF4B69A6EB07080F608B60B8F14B
:10220000000F9ADD43463A46216A2846A66AB0473F
:10221000002807DCA38943F04003A3814FF0FF307F
:10222000BDE8F0810744A8EB0008E8E70100402082
:1022300038B50B6905460C46DBB118B183690BB99B
:1022400000F060F80C4B9C4209D16C68B4F90C307A
:102250007BB121462846BDE83840FFF761BF074BF8
:102260009C4201D1AC68F1E7054B9C4208BFEC6889
:10227000ECE7002038BD00BF582F0008782F000879
:10228000382F0008014900F0A9B800BF312200082A
:10229000002310B504460360436083608181436678
:1022A000C281036143618361194608225C30FFF7F4
:1022B0003DFD054B24626362044BA362044BE36261
:1022C000044B236310BD00BF112C0008332C000801
:1022D0006B2C00088F2C000870B568254A1E5543EA
:1022E0000E4605F1740100F04FF9044640B100219B
:1022F00080E842000C30A06005F16802FFF716FD8F
:10230000204670BD836910B5044633BB8364C36443
:102310000365124B124A1B688262984204BF012374
:10232000836100F01FF86060204600F01BF8A06099
:10233000204600F017F80022E06004216068FFF7F3
:10234000A7FF01220921A068FFF7A2FF02221221A4
:10235000E068FFF79DFF0123A36110BD342F000843
:1023600085220008F8B51C4B07461E68B36913B9EF
:102370003046FFF7C7FF4836B4687368013B03D5A2
:10238000336833B13668F7E7B4F90C506DB168348F
:10239000F4E704213846FFF79FFF30600028F1D1B1
:1023A0000C2304463B602046F8BD4FF6FF73E381E3
:1023B00001236566A3812560A5606560256165616F
:1023C000A5610822294604F15C00FFF7AFFC6563B4
:1023D000A563A564E564E6E7342F00082DE9F8431A
:1023E00080468946002600F1480414B93046BDE80D
:1023F000F883A5686768013F01D52468F5E7AB89D4
:10240000012B07D9B5F90E30013303D029464046D8
:10241000C84706436835EEE770B50E46B1F90E10B1
:1024200090B0002914461D4607DA00232B60B389BB
:102430001A0610D44FF480630EE001AA00F04EFC9F
:102440000028F2DB029A02F47042A2F500535A42CD
:102450005A412A60EEE740230020236010B070BD8F
:102460008B8973B59D0706460C4607D504F14703D3
:10247000236023610123636102B070BD01AB6A4632
:10248000FFF7CAFF00990546304600F07DF848B9CD
:10249000B4F90C309A05EFD423F0030343F00203A0
:1024A000A381E3E70D4BB362A389206043F080036F
:1024B000A381009B20616361019B5BB1B4F90E10A5
:1024C000304600F01DFC28B1A38923F0030343F03C
:1024D0000103A381A3891D43A581CDE785220008BF
:1024E000024B0146186800F04FB800BF10000020F2
:1024F00038B50546002943D051F8043C0C1F002B89
:10250000B8BFE41800F02CFC1E4A1368104633B91B
:10251000636014602846BDE8384000F022BCA34246
:102520000BD921686218934201BF1A685B68521880
:10253000226063600460EDE713465A680AB1A24264
:10254000FAD919685818A0420BD1206801445818CC
:1025500082421960DED110685268014419605A60E5
:10256000D8E702D90C232B60D4E7206821188A42CF
:1025700001BF116852680918216062605C60C9E798
:1025800038BD00BFC400002070B5CD1C25F0030588
:1025900008350C2D38BF0C25002D064601DBA9425D
:1025A00003D90C233360002070BD00F0D9FB234A0F
:1025B0001468214691B9224C23681BB9304600F0BB
:1025C00017FB20602946304600F012FB431C26D141
:1025D0000C233046336000F0C4FBE4E70B685B1B60
:1025E0001AD40B2B0FD90B60CC18CD50304600F00D
:1025F000B8FB04F10B00231D20F00700C31A1BD009
:102600005A42E25070BD8C420BBF63684B68136046
:10261000636018BF0C46E9E70C464968CAE7C41C6A
:1026200024F00304A04205D0211A304600F0E0FA5D
:102630000130CDD02560D9E770BD00BFC4000020B7
:10264000C8000020936810B4013B002B936008DAA7
:102650009469A34202DBCBB20A2B02D110BCFFF774
:102660009FBC1368581C10601970C8B210BC70472A
:10267000F8B506460F461446D518AC4201D10020E5
:1026800007E03A4614F8011B3046FFF7DBFF431C16
:10269000F3D1F8BD2DE9F04F9DB00C4617460393DA
:1026A000064618B183690BB9FFF72CFE7C4B9C42A0
:1026B00057D17468A38918075DD52369002B5AD0B8
:1026C0000023099320238DF8293030234FF0010B8C
:1026D0008DF82A30B846454615F8013B002B55D1F8
:1026E000B8EB070A0BD053463A4621463046FFF76F
:1026F000BFFF013000F0C480099B5344099398F850
:102700000030002B00F0BC8000234FF0FF32049318
:102710000793059206938DF853301A930522297872
:10272000604800F00FFB05F10108049B002831D13F
:10273000D90644BF20228DF853201A0744BF2B220C
:102740008DF853202A782A2A2CD000210A20079AB3
:10275000A84698F800300135303B092B6DD971B38C
:1027600026E0514B9C4201D1B468A3E74F4B9C42F9
:1027700008BFF4689EE721463046FFF763FC002857
:102780009ED04FF0FF301DB0BDE8F08F252BA7D0B5
:10279000A846A0E7434A4546801A0BFA00F01843C2
:1027A0000490BBE7039A111D12680391002A01DB14
:1027B000079204E0524243F002030792049398F810
:1027C00000302E2B10D198F8013008F101012A2B8E
:1027D00037D1039B08F102081A1D1B680392002BD6
:1027E000B8BF4FF0FF330593314D032298F8001026
:1027F000284600F0A7FA40B14023401B03FA00F03E
:10280000049B08F101080343049398F80010062282
:10281000284808F101078DF8281000F093FA0028E5
:1028200034D0254B03BB039B073323F00703083346
:102830000393099B4B4409934CE700FB02320121AF
:1028400086E700230A2518460593884698F8002055
:102850000131303A092A03D9002BC5D00590C3E7CE
:1028600005FB00200123F0E703AB00932246134B46
:1028700004A93046AFF30080B0F1FF3F8146D8D1C4
:10288000A3895B063FF57DAF09987CE703AB009316
:1028900022460A4B04A9304600F08AF8ECE700BF54
:1028A000582F0008982F0008782F0008382F0008AC
:1028B0009E2F0008A22F00080000000071260008CB
:1028C0002DE9F04791461F468A680B6906469342F8
:1028D000B8BF1346C9F8003091F843200C46DDF824
:1028E000208012B10133C9F800302368990642BF35
:1028F000D9F800300233C9F80030256815F0060514
:1029000007D104F1190AE368D9F800209B1A9D4207
:102910002ADB94F843302268003318BF0123920663
:102920002FD404F1430239463046C047013022D04B
:102930002368E56803F00603042B18BF0025D9F8C7
:1029400000204FF0000908BFAD1AA368226908BF34
:1029500025EAE5759342C4BF9B1AED181A344D451C
:102960001BD10020BDE8F08701235246394630468E
:10297000C047013003D14FF0FF30BDE8F08701358B
:10298000C1E73020E11881F843005A1C94F8451043
:102990002244023382F84310C3E70123224639461A
:1029A0003046C0470130E6D009F10109D7E7000001
:1029B0002DE9F04317460A7E85B06E2A98460646F2
:1029C0000C460C9B01F1430E00F0BC801AD8632A20
:1029D0002ED00AD8002A00F0C880582A00F08A8039
:1029E00004F1420584F842202AE0642A01D0692AD1
:1029F000F6D121681A6811F0800F23D0111D1960DB
:102A0000136827E0732A00F0B48008D86F2A2AD010
:102A1000702AE5D10A6842F020020A6003E0752AB4
:102A200021D0782ADCD178226F4984F8452064E0EF
:102A30001A6801F14205111D1960136884F84230CB
:102A40000123A3E011F0400F02F104011960D7D077
:102A5000B2F90030002B03DA2D225B4284F84320C8
:102A600062490A2217E02068196810F0800F03D02D
:102A7000081D18600B6806E010F0400F01F104001B
:102A80001860F7D00B886F2A14BF0A220822574912
:102A9000002084F843006568002DA560C0F29C808A
:102AA000206820F004002060002B3FD1002D40F072
:102AB00095807546082A0BD12368DA0708D5236963
:102AC00062689A42DEBF302305F8013C05F1FF350C
:102AD000AEEB05032361CDF800803B4603AA2146F7
:102AE0003046FFF7EDFE013055D14FF0FF3005B015
:102AF000BDE8F08381F845203C492268186812F04F
:102B0000800F00F104051D6001D0036802E0550646
:102B1000FBD50388D00744BF42F0200222601BB9D6
:102B2000226822F0200222601022B1E77546B3FB32
:102B3000F2F002FB1033CB5C05F8013D03460028A0
:102B4000F5D1B7E708681A6810F0800F496904D01A
:102B5000101D18601368196007E010F0400F02F1B3
:102B6000040018601368F6D01980002375462361AD
:102B7000B1E71A68111D19601568002162682846BE
:102B800000F0E0F808B1401B606063682361002337
:102B900084F843309FE723692A4639463046C047C8
:102BA0000130A2D023689B0707D5002504F119093D
:102BB000E368039A9B1A9D4205DBE068039B9842F9
:102BC000B8BF184693E701234A4639463046C04706
:102BD00001308AD00135EBE7002BA7D10B7804F147
:102BE000420584F8423065E7BA2F0008A92F000893
:102BF00038B50023054C05460846236000F0ECF884
:102C0000431C02D1236803B12B6038BD8802002029
:102C100010B50C46B1F90E1000F0A4F80028ABBFB7
:102C2000636DA3891B1823F48053ACBF6365A38134
:102C300010BD2DE9F0411F468B890546DB050C468A
:102C4000164605D502230022B1F90E1000F068F8EF
:102C5000A389324623F48053A381B4F90E103B4676
:102C60002846BDE8F04100F017B810B50C46B1F9A0
:102C70000E1000F055F8431CA38915BF606523F4BE
:102C8000805343F48053A38118BFA38110BDB1F9D1
:102C90000E1000F013B8000038B50546084611467E
:102CA0000022054C22601A46FEF7C8FC431C02D1E4
:102CB000236803B12B6038BD8802002038B500239B
:102CC000054C05460846236000F05EF8431C02D11F
:102CD000236803B12B6038BD8802002038B500237B
:102CE000064C054608461146236000F055F8431C83
:102CF00002D1236803B12B6038BD00BF88020020D9
:102D000038B50023054C05460846236000F04CF812
:102D1000431C02D1236803B12B6038BD8802002018
:102D200038B50546084611460022054C22601A4671
:102D300000F042F8431C02D1236803B12B6038BD78
:102D40008802002010B5C9B202449042034601D166
:102D5000002010BD1C7801308C42F6D1184610BD01
:102D60007047704738B50546084611460022054CA5
:102D700022601A4600F028F8431C02D1236803B1F0
:102D80002B6038BD880200205822024B4FF0FF30E4
:102D90001A607047880200205822024B4FF0FF3023
:102DA0001A607047880200205822024B00201A60E7
:102DB000704700BF880200205822024B4FF0FF30BE
:102DC0001A607047880200205822024B4FF0FF30F3
:102DD0001A60704788020020044B0246196809B93E
:102DE00003491960186802441A607047CC0000203B
:102DF0008C020020F8B500BFF8BC08BC9E467047A6
:0C2E0000F8B500BFF8BC08BC9E46704747
:102E0C0002030405060708090A0B0C0D0E0F10101F
:102E1C000102030405060708090A0B0C0D0E0F101E
:102E2C00BE110200BEBE0B0200EB25303278200032
:102E3C00436865636B2053756D206572726F7220E9
:102E4C000075706461746520436F6D706C6574659A
:102E5C00200025303878203A2025303258200A00BE
:102E6C0048414C204E4F54204F4B2000457261730B
:102E7C0065204661696C6564200D00626F6F74207B
:102E8C006C6F61646572207374617274006A756D25
:102E9C007021002A2A2A2A2A2A2A2A2A2A2A2A2A73
:102EAC002A2A2A2A2A2A2A2A2A2A2A2A2A2A2A2A76
:102EBC002A2A2A2A2A2A2A2A2A2A2A0D0052474250
:102ECC002050726F6A6563740D0031343A31353AB3
:102EDC0033300041707220203120323031390042C1
:102EEC0075696C642061742025732025730D0A00AC
:102EFC00436F7079726967687420286329203230B7
:102F0C0031392E20424C554543454C4C0D000000A8
:102F1C00000000000000010203040607080900007D
:102F2C000000010203040000140000200000000057
:102F3C000000000000000000000000000000000085
:102F4C000000000000000000000000000000000075
:102F5C000000000000000000000000000000000065
:102F6C000000000000000000000000000000000055
:102F7C000000000000000000000000000000000045
:102F8C00000000000000000000000000232D302B8A
:102F9C002000686C4C00656667454647003031324E
:102FAC0033343536373839414243444546003031A5
:102FBC003233343536373839616263646566000004
:042FCC00F501000803
:042FD000D101000823
:102FD40001000000100000000040000800366E01EF
:102FE4001400002000000000582F0008782F00086B
:102FF400382F00080000000000000000000000005E
:1030040000000000000000000000000000000000BC
:1030140000000000000000000000000000000000AC
:10302400000000000000000000000000000000009C
:10303400000000000000000000000000000000008C
:043044000000000088
:0400000508001C993A
:00000001FF
